 prefs

 Timestamp is ffffffff (Sun Feb  7 06:28:15 2106)

 Preferred load address is 10000000

 Start         Length     Name                   Class
 0001:00000000 00001290H .text$mn                CODE
 0002:00000000 000000acH .idata$5                DATA
 0002:000000ac 00000004H .00cfg                  DATA
 0002:000000b0 00000004H .CRT$XCA                DATA
 0002:000000b4 00000004H .CRT$XCZ                DATA
 0002:000000b8 00000004H .CRT$XIA                DATA
 0002:000000bc 00000004H .CRT$XIZ                DATA
 0002:000000c0 00000004H .CRT$XPA                DATA
 0002:000000c4 00000004H .CRT$XPZ                DATA
 0002:000000c8 00000004H .CRT$XTA                DATA
 0002:000000cc 00000004H .CRT$XTZ                DATA
 0002:000000d0 00000000H .gfids$y                DATA
 0002:000000d0 00000158H .rdata                  DATA
 0002:00000228 00000004H .rdata$sxdata           DATA
 0002:0000022c 00000284H .rdata$zzzdbg           DATA
 0002:000004b0 00000004H .rtc$IAA                DATA
 0002:000004b4 00000004H .rtc$IZZ                DATA
 0002:000004b8 00000004H .rtc$TAA                DATA
 0002:000004bc 00000004H .rtc$TZZ                DATA
 0002:000004c0 00000090H .xdata$x                DATA
 0002:00000550 00000368H .edata                  DATA
 0002:000008b8 00000078H .idata$2                DATA
 0002:00000930 00000014H .idata$3                DATA
 0002:00000944 000000acH .idata$4                DATA
 0002:000009f0 00000374H .idata$6                DATA
 0003:00000000 00000018H .data                   DATA
 0003:00000018 00000374H .bss                    DATA
 0004:00000000 00000060H .rsrc$01                DATA
 0004:00000060 00000318H .rsrc$02                DATA

  Address         Publics by Value              Rva+Base       Lib:Object

 0000:00000000       ___arm64x_native_entrypoint 00000000     <absolute>
 0000:00000000       ___hybrid_code_map         00000000     <absolute>
 0000:00000000       ___guard_fids_table        00000000     <absolute>
 0000:00000000       ___arm64x_redirection_metadata_count 00000000     <absolute>
 0000:00000000       ___hybrid_code_map_count   00000000     <absolute>
 0000:00000000       ___guard_longjmp_table     00000000     <absolute>
 0000:00000000       ___guard_fids_count        00000000     <absolute>
 0000:00000000       ___x64_code_ranges_to_entry_points 00000000     <absolute>
 0000:00000000       ___guard_longjmp_count     00000000     <absolute>
 0000:00000000       ___AbsoluteZero            00000000     <absolute>
 0000:00000000       ___guard_iat_table         00000000     <absolute>
 0000:00000000       ___hybrid_auxiliary_iat    00000000     <absolute>
 0000:00000000       ___guard_eh_cont_count     00000000     <absolute>
 0000:00000000       ___arm64x_redirection_metadata 00000000     <absolute>
 0000:00000000       ___volatile_metadata       00000000     <absolute>
 0000:00000000       ___dynamic_value_reloc_table 00000000     <absolute>
 0000:00000000       ___arm64x_extra_rfe_table_size 00000000     <absolute>
 0000:00000000       ___arm64x_extra_rfe_table  00000000     <absolute>
 0000:00000000       ___enclave_config          00000000     <absolute>
 0000:00000000       ___x64_code_ranges_to_entry_points_count 00000000     <absolute>
 0000:00000000       ___guard_iat_count         00000000     <absolute>
 0000:00000000       ___guard_eh_cont_table     00000000     <absolute>
 0000:00000001       ___safe_se_handler_count   00000001     <absolute>
 0000:00000100       ___guard_flags             00000100     <absolute>
 0000:00000000       ___ImageBase               10000000     <linker-defined>
 0001:00000000       _Java_java_util_prefs_WindowsPreferences_WindowsRegCloseKey@16 10001000 f   WindowsPreferences.obj
 0001:0000000d       _Java_java_util_prefs_WindowsPreferences_WindowsRegCreateKeyEx@20 1000100d f   WindowsPreferences.obj
 0001:000000db       _Java_java_util_prefs_WindowsPreferences_WindowsRegDeleteKey@20 100010db f   WindowsPreferences.obj
 0001:00000121       _Java_java_util_prefs_WindowsPreferences_WindowsRegDeleteValue@20 10001121 f   WindowsPreferences.obj
 0001:0000016e       _Java_java_util_prefs_WindowsPreferences_WindowsRegEnumKeyEx@24 1000116e f   WindowsPreferences.obj
 0001:000001f6       _Java_java_util_prefs_WindowsPreferences_WindowsRegEnumValue@24 100011f6 f   WindowsPreferences.obj
 0001:0000027e       _Java_java_util_prefs_WindowsPreferences_WindowsRegFlushKey@16 1000127e f   WindowsPreferences.obj
 0001:0000028b       _Java_java_util_prefs_WindowsPreferences_WindowsRegOpenKey@24 1000128b f   WindowsPreferences.obj
 0001:0000031d       _Java_java_util_prefs_WindowsPreferences_WindowsRegQueryInfoKey@16 1000131d f   WindowsPreferences.obj
 0001:000003de       _Java_java_util_prefs_WindowsPreferences_WindowsRegQueryValueEx@20 100013de f   WindowsPreferences.obj
 0001:000004c9       _Java_java_util_prefs_WindowsPreferences_WindowsRegSetValueEx@24 100014c9 f   WindowsPreferences.obj
 0001:00000568       _JNU_ThrowOutOfMemoryError@8 10001568 f   java:java.dll
 0001:0000056e       @__security_check_cookie@4 1000156e f   MSVCRT:secchk.obj
 0001:000008bf       __DllMainCRTStartup@12     100018bf f   MSVCRT:dll_dllmain.obj
 0001:000008e2       ___raise_securityfailure   100018e2 f   MSVCRT:gs_report.obj
 0001:0000090a       ___report_gsfailure        1000190a f   MSVCRT:gs_report.obj
 0001:00000a50       ___security_init_cookie    10001a50 f   MSVCRT:gs_support.obj
 0001:00000a9b       _DllMain@12                10001a9b f   MSVCRT:dll_dllmain_stub.obj
 0001:00000abd       ?__scrt_initialize_type_info@@YAXXZ 10001abd f   MSVCRT:tncleanup.obj
 0001:00000ac9       ?__scrt_uninitialize_type_info@@YAXXZ 10001ac9 f   MSVCRT:tncleanup.obj
 0001:00000ad5       ___local_stdio_printf_options 10001ad5 f i MSVCRT:default_local_stdio_options.obj
 0001:00000adb       ___local_stdio_scanf_options 10001adb f i MSVCRT:default_local_stdio_options.obj
 0001:00000ae1       ___scrt_initialize_default_local_stdio_options 10001ae1 f   MSVCRT:default_local_stdio_options.obj
 0001:00000b42       ___scrt_acquire_startup_lock 10001b42 f   MSVCRT:utility.obj
 0001:00000b74       ___scrt_dllmain_after_initialize_c 10001b74 f   MSVCRT:utility.obj
 0001:00000b9f       ___scrt_dllmain_before_initialize_c 10001b9f f   MSVCRT:utility.obj
 0001:00000bad       ___scrt_dllmain_crt_thread_attach 10001bad f   MSVCRT:utility.obj
 0001:00000bcc       ___scrt_dllmain_crt_thread_detach 10001bcc f   MSVCRT:utility.obj
 0001:00000bd9       ___scrt_dllmain_exception_filter 10001bd9 f   MSVCRT:utility.obj
 0001:00000c0d       ___scrt_dllmain_uninitialize_c 10001c0d f   MSVCRT:utility.obj
 0001:00000c30       ___scrt_dllmain_uninitialize_critical 10001c30 f   MSVCRT:utility.obj
 0001:00000c3d       ___scrt_initialize_crt     10001c3d f   MSVCRT:utility.obj
 0001:00000c76       ___scrt_initialize_onexit_tables 10001c76 f   MSVCRT:utility.obj
 0001:00000cfd       ___scrt_is_nonwritable_in_current_image 10001cfd f   MSVCRT:utility.obj
 0001:00000d91       ___scrt_release_startup_lock 10001d91 f   MSVCRT:utility.obj
 0001:00000dae       ___scrt_uninitialize_crt   10001dae f   MSVCRT:utility.obj
 0001:00000dd6       ___scrt_get_dyn_tls_init_callback 10001dd6 f   MSVCRT:dyn_tls_init.obj
 0001:00000ddc       ___scrt_fastfail           10001ddc f   MSVCRT:utility_desktop.obj
 0001:00000ef6       __crt_debugger_hook        10001ef6 f   MSVCRT:utility_desktop.obj
 0001:00000efe       __RTC_Initialize           10001efe f   MSVCRT:initsect.obj
 0001:00000f2a       __RTC_Terminate            10001f2a f   MSVCRT:initsect.obj
 0001:00000f60       __SEH_prolog4              10001f60 f   MSVCRT:sehprolg4.obj
 0001:00000fa4       __SEH_epilog4              10001fa4 f   MSVCRT:sehprolg4.obj
 0001:00000fb8       __except_handler4          10001fb8 f   MSVCRT:chandler4gs.obj
 0001:00000fe7       @_guard_check_icall_nop@4  10001fe7 f i MSVCRT:guard_support.obj
 0001:00000fea       ___isa_available_init      10001fea f   MSVCRT:cpu_disp.obj
 0001:000011ba       __get_startup_argv_mode    100021ba f   MSVCRT:argv_mode.obj
 0001:000011be       ___scrt_is_ucrt_dll_in_use 100021be f   MSVCRT:ucrt_detection.obj
 0001:000011ca       _IsProcessorFeaturePresent@4 100021ca f   kernel32:KERNEL32.dll
 0001:000011d0       ___std_type_info_destroy_list 100021d0 f   vcruntime:VCRUNTIME140.dll
 0001:000011d6       _memset                    100021d6 f   vcruntime:VCRUNTIME140.dll
 0001:000011dc       __except_handler4_common   100021dc f   vcruntime:VCRUNTIME140.dll
 0001:000011e2       __initterm                 100021e2 f   ucrt:api-ms-win-crt-runtime-l1-1-0.dll
 0001:000011e8       __initterm_e               100021e8 f   ucrt:api-ms-win-crt-runtime-l1-1-0.dll
 0001:000011ee       __seh_filter_dll           100021ee f   ucrt:api-ms-win-crt-runtime-l1-1-0.dll
 0001:000011f4       __configure_narrow_argv    100021f4 f   ucrt:api-ms-win-crt-runtime-l1-1-0.dll
 0001:000011fa       __initialize_narrow_environment 100021fa f   ucrt:api-ms-win-crt-runtime-l1-1-0.dll
 0001:00001200       __initialize_onexit_table  10002200 f   ucrt:api-ms-win-crt-runtime-l1-1-0.dll
 0001:00001206       __execute_onexit_table     10002206 f   ucrt:api-ms-win-crt-runtime-l1-1-0.dll
 0001:0000120c       __cexit                    1000220c f   ucrt:api-ms-win-crt-runtime-l1-1-0.dll
 0001:00001212       ___scrt_stub_for_acrt_thread_attach 10002212 f   MSVCRT:ucrt_stubs.obj
 0001:00001212       ___scrt_stub_for_acrt_initialize 10002212 f   MSVCRT:ucrt_stubs.obj
 0001:00001212       ___acrt_uninitialize       10002212 f   MSVCRT:ucrt_stubs.obj
 0001:00001212       ___acrt_thread_attach      10002212 f   MSVCRT:ucrt_stubs.obj
 0001:00001212       ___scrt_stub_for_acrt_thread_detach 10002212 f   MSVCRT:ucrt_stubs.obj
 0001:00001212       ___vcrt_thread_attach      10002212 f   MSVCRT:ucrt_stubs.obj
 0001:00001212       ___vcrt_uninitialize_critical 10002212 f   MSVCRT:ucrt_stubs.obj
 0001:00001212       ___vcrt_uninitialize       10002212 f   MSVCRT:ucrt_stubs.obj
 0001:00001212       ___acrt_initialize         10002212 f   MSVCRT:ucrt_stubs.obj
 0001:00001212       ___scrt_stub_for_acrt_uninitialize_critical 10002212 f   MSVCRT:ucrt_stubs.obj
 0001:00001212       ___vcrt_thread_detach      10002212 f   MSVCRT:ucrt_stubs.obj
 0001:00001212       ___acrt_uninitialize_critical 10002212 f   MSVCRT:ucrt_stubs.obj
 0001:00001212       ___scrt_stub_for_acrt_uninitialize 10002212 f   MSVCRT:ucrt_stubs.obj
 0001:00001212       ___vcrt_initialize         10002212 f   MSVCRT:ucrt_stubs.obj
 0001:00001212       ___acrt_thread_detach      10002212 f   MSVCRT:ucrt_stubs.obj
 0001:00001215       __is_c_termination_complete 10002215 f   MSVCRT:ucrt_stubs.obj
 0001:00001215       ___scrt_stub_for_is_c_termination_complete 10002215 f   MSVCRT:ucrt_stubs.obj
 0001:00001218       __filter_x86_sse2_floating_point_exception 10002218 f   MSVCRT:x86_exception_filter.obj
 0001:00001218       __filter_x86_sse2_floating_point_exception_default 10002218 f   MSVCRT:x86_exception_filter.obj
 0002:00000000       __imp__RegCloseKey@4       10003000     advapi32:ADVAPI32.dll
 0002:00000004       __imp__RegCreateKeyExA@36  10003004     advapi32:ADVAPI32.dll
 0002:00000008       __imp__RegDeleteKeyA@8     10003008     advapi32:ADVAPI32.dll
 0002:0000000c       __imp__RegDeleteValueA@8   1000300c     advapi32:ADVAPI32.dll
 0002:00000010       __imp__RegEnumKeyExA@32    10003010     advapi32:ADVAPI32.dll
 0002:00000014       __imp__RegEnumValueA@32    10003014     advapi32:ADVAPI32.dll
 0002:00000018       __imp__RegFlushKey@4       10003018     advapi32:ADVAPI32.dll
 0002:0000001c       __imp__RegOpenKeyExA@20    1000301c     advapi32:ADVAPI32.dll
 0002:00000020       __imp__RegQueryInfoKeyA@48 10003020     advapi32:ADVAPI32.dll
 0002:00000024       __imp__RegQueryValueExA@24 10003024     advapi32:ADVAPI32.dll
 0002:00000028       __imp__RegSetValueExA@24   10003028     advapi32:ADVAPI32.dll
 0002:0000002c       \177ADVAPI32_NULL_THUNK_DATA 1000302c     advapi32:ADVAPI32.dll
 0002:00000030       __imp__UnhandledExceptionFilter@4 10003030     kernel32:KERNEL32.dll
 0002:00000034       __imp__SetUnhandledExceptionFilter@4 10003034     kernel32:KERNEL32.dll
 0002:00000038       __imp__GetCurrentProcess@0 10003038     kernel32:KERNEL32.dll
 0002:0000003c       __imp__TerminateProcess@8  1000303c     kernel32:KERNEL32.dll
 0002:00000040       __imp__IsProcessorFeaturePresent@4 10003040     kernel32:KERNEL32.dll
 0002:00000044       __imp__QueryPerformanceCounter@4 10003044     kernel32:KERNEL32.dll
 0002:00000048       __imp__GetCurrentProcessId@0 10003048     kernel32:KERNEL32.dll
 0002:0000004c       __imp__GetCurrentThreadId@0 1000304c     kernel32:KERNEL32.dll
 0002:00000050       __imp__GetSystemTimeAsFileTime@4 10003050     kernel32:KERNEL32.dll
 0002:00000054       __imp__DisableThreadLibraryCalls@4 10003054     kernel32:KERNEL32.dll
 0002:00000058       __imp__InitializeSListHead@4 10003058     kernel32:KERNEL32.dll
 0002:0000005c       __imp__IsDebuggerPresent@0 1000305c     kernel32:KERNEL32.dll
 0002:00000060       \177KERNEL32_NULL_THUNK_DATA 10003060     kernel32:KERNEL32.dll
 0002:00000064       __imp___except_handler4_common 10003064     vcruntime:VCRUNTIME140.dll
 0002:00000068       __imp____std_type_info_destroy_list 10003068     vcruntime:VCRUNTIME140.dll
 0002:0000006c       __imp__memset              1000306c     vcruntime:VCRUNTIME140.dll
 0002:00000070       \177VCRUNTIME140_NULL_THUNK_DATA 10003070     vcruntime:VCRUNTIME140.dll
 0002:00000074       __imp__free                10003074     ucrt:api-ms-win-crt-heap-l1-1-0.dll
 0002:00000078       __imp__malloc              10003078     ucrt:api-ms-win-crt-heap-l1-1-0.dll
 0002:0000007c       \177api-ms-win-crt-heap-l1-1-0_NULL_THUNK_DATA 1000307c     ucrt:api-ms-win-crt-heap-l1-1-0.dll
 0002:00000080       __imp___initterm_e         10003080     ucrt:api-ms-win-crt-runtime-l1-1-0.dll
 0002:00000084       __imp___initterm           10003084     ucrt:api-ms-win-crt-runtime-l1-1-0.dll
 0002:00000088       __imp___cexit              10003088     ucrt:api-ms-win-crt-runtime-l1-1-0.dll
 0002:0000008c       __imp___seh_filter_dll     1000308c     ucrt:api-ms-win-crt-runtime-l1-1-0.dll
 0002:00000090       __imp___configure_narrow_argv 10003090     ucrt:api-ms-win-crt-runtime-l1-1-0.dll
 0002:00000094       __imp___initialize_narrow_environment 10003094     ucrt:api-ms-win-crt-runtime-l1-1-0.dll
 0002:00000098       __imp___initialize_onexit_table 10003098     ucrt:api-ms-win-crt-runtime-l1-1-0.dll
 0002:0000009c       __imp___execute_onexit_table 1000309c     ucrt:api-ms-win-crt-runtime-l1-1-0.dll
 0002:000000a0       \177api-ms-win-crt-runtime-l1-1-0_NULL_THUNK_DATA 100030a0     ucrt:api-ms-win-crt-runtime-l1-1-0.dll
 0002:000000a4       __imp__JNU_ThrowOutOfMemoryError@8 100030a4     java:java.dll
 0002:000000a8       \177java_NULL_THUNK_DATA   100030a8     java:java.dll
 0002:000000ac       ___guard_check_icall_fptr  100030ac     MSVCRT:guard_support.obj
 0002:000000b0       ___xc_a                    100030b0     MSVCRT:initializers.obj
 0002:000000b4       ___xc_z                    100030b4     MSVCRT:initializers.obj
 0002:000000b8       ___xi_a                    100030b8     MSVCRT:initializers.obj
 0002:000000bc       ___xi_z                    100030bc     MSVCRT:initializers.obj
 0002:000000c0       ___xp_a                    100030c0     MSVCRT:initializers.obj
 0002:000000c4       ___xp_z                    100030c4     MSVCRT:initializers.obj
 0002:000000c8       ___xt_a                    100030c8     MSVCRT:initializers.obj
 0002:000000cc       ___xt_z                    100030cc     MSVCRT:initializers.obj
 0002:000000d0       ??_C@_0CA@NIIGFDJD@native?5memory?5allocation?5failed@ 100030d0     WindowsPreferences.obj
 0002:000000f0       __pRawDllMain              100030f0     MSVCRT:dll_dllmain.obj
 0002:000000f0       __pDefaultRawDllMain       100030f0     MSVCRT:dll_dllmain.obj
 0002:00000170       __load_config_used         10003170     MSVCRT:loadcfg.obj
 0002:00000228       ___safe_se_handler_table   10003228     <linker-defined>
 0002:000004b0       ___rtc_iaa                 100034b0     MSVCRT:initsect.obj
 0002:000004b4       ___rtc_izz                 100034b4     MSVCRT:initsect.obj
 0002:000004b8       ___rtc_taa                 100034b8     MSVCRT:initsect.obj
 0002:000004bc       ___rtc_tzz                 100034bc     MSVCRT:initsect.obj
 0002:000008b8       __IMPORT_DESCRIPTOR_ADVAPI32 100038b8     advapi32:ADVAPI32.dll
 0002:000008cc       __IMPORT_DESCRIPTOR_java   100038cc     java:java.dll
 0002:000008e0       __IMPORT_DESCRIPTOR_KERNEL32 100038e0     kernel32:KERNEL32.dll
 0002:000008f4       __IMPORT_DESCRIPTOR_VCRUNTIME140 100038f4     vcruntime:VCRUNTIME140.dll
 0002:00000908       __IMPORT_DESCRIPTOR_api-ms-win-crt-heap-l1-1-0 10003908     ucrt:api-ms-win-crt-heap-l1-1-0.dll
 0002:0000091c       __IMPORT_DESCRIPTOR_api-ms-win-crt-runtime-l1-1-0 1000391c     ucrt:api-ms-win-crt-runtime-l1-1-0.dll
 0002:00000930       __NULL_IMPORT_DESCRIPTOR   10003930     advapi32:ADVAPI32.dll
 0003:00000000       ___security_cookie_complement 10004000     MSVCRT:gs_cookie.obj
 0003:00000004       ___security_cookie         10004004     MSVCRT:gs_cookie.obj
 0003:00000008       ___scrt_native_dllmain_reason 10004008     MSVCRT:utility.obj
 0003:00000010       ___isa_enabled             10004010     MSVCRT:cpu_disp.obj
 0003:00000014       ___scrt_ucrt_dll_is_in_use 10004014     MSVCRT:ucrt_stubs.obj
 0003:00000340       ?__type_info_root_node@@3U__type_info_node@@A 10004340     MSVCRT:tncleanup.obj
 0003:00000348       ?_OptionsStorage@?1??__local_stdio_printf_options@@9@4_KA 10004348     MSVCRT:default_local_stdio_options.obj
 0003:00000350       ?_OptionsStorage@?1??__local_stdio_scanf_options@@9@4_KA 10004350     MSVCRT:default_local_stdio_options.obj
 0003:00000358       ___scrt_current_native_startup_state 10004358     MSVCRT:utility.obj
 0003:0000035c       ___scrt_native_startup_lock 1000435c     MSVCRT:utility.obj
 0003:0000037c       ___scrt_debugger_hook_flag 1000437c     MSVCRT:utility_desktop.obj
 0003:00000380       ___isa_available           10004380     MSVCRT:cpu_disp.obj
 0003:00000384       ___favor                   10004384     MSVCRT:cpu_disp.obj
 0003:00000388       ___dyn_tls_init_callback   10004388     <common>

 entry point at        0001:000008bf

 Static symbols

 0000:ffff9000       .debug$S                   10000000     prefs.exp
 0000:ffff9000       .debug$S                   10000000     vcruntime:VCRUNTIME140.dll
 0000:ffff9000       .debug$S                   10000000     vcruntime:VCRUNTIME140.dll
 0000:ffff9000       .debug$S                   10000000     vcruntime:VCRUNTIME140.dll
 0000:ffff9000       .debug$S                   10000000     vcruntime:VCRUNTIME140.dll
 0000:ffff9000       .debug$S                   10000000     vcruntime:VCRUNTIME140.dll
 0000:ffff9000       .debug$S                   10000000     ucrt:api-ms-win-crt-heap-l1-1-0.dll
 0000:ffff9000       .debug$S                   10000000     ucrt:api-ms-win-crt-heap-l1-1-0.dll
 0000:ffff9000       .debug$S                   10000000     ucrt:api-ms-win-crt-runtime-l1-1-0.dll
 0000:ffff9000       .debug$S                   10000000     ucrt:api-ms-win-crt-runtime-l1-1-0.dll
 0000:ffff9000       .debug$S                   10000000     ucrt:api-ms-win-crt-runtime-l1-1-0.dll
 0000:ffff9000       .debug$S                   10000000     ucrt:api-ms-win-crt-runtime-l1-1-0.dll
 0000:ffff9000       .debug$S                   10000000     ucrt:api-ms-win-crt-runtime-l1-1-0.dll
 0000:ffff9000       .debug$S                   10000000     ucrt:api-ms-win-crt-runtime-l1-1-0.dll
 0000:ffff9000       .debug$S                   10000000     ucrt:api-ms-win-crt-runtime-l1-1-0.dll
 0000:ffff9000       .debug$S                   10000000     ucrt:api-ms-win-crt-runtime-l1-1-0.dll
 0000:ffff9000       .debug$S                   10000000     ucrt:api-ms-win-crt-runtime-l1-1-0.dll
 0000:ffff9000       .debug$S                   10000000     ucrt:api-ms-win-crt-runtime-l1-1-0.dll
 0000:ffff9000       .debug$S                   10000000     ucrt:api-ms-win-crt-runtime-l1-1-0.dll
 0000:ffff9000       .debug$S                   10000000     ucrt:api-ms-win-crt-runtime-l1-1-0.dll
 0000:ffff9000       .debug$S                   10000000     advapi32:ADVAPI32.dll
 0000:ffff9000       .debug$S                   10000000     advapi32:ADVAPI32.dll
 0000:ffff9000       .debug$S                   10000000     advapi32:ADVAPI32.dll
 0000:ffff9000       .debug$S                   10000000     advapi32:ADVAPI32.dll
 0000:ffff9000       .debug$S                   10000000     advapi32:ADVAPI32.dll
 0000:ffff9000       .debug$S                   10000000     advapi32:ADVAPI32.dll
 0000:ffff9000       .debug$S                   10000000     advapi32:ADVAPI32.dll
 0000:ffff9000       .debug$S                   10000000     advapi32:ADVAPI32.dll
 0000:ffff9000       .debug$S                   10000000     advapi32:ADVAPI32.dll
 0000:ffff9000       .debug$S                   10000000     advapi32:ADVAPI32.dll
 0000:ffff9000       .debug$S                   10000000     advapi32:ADVAPI32.dll
 0000:ffff9000       .debug$S                   10000000     kernel32:KERNEL32.dll
 0000:ffff9000       .debug$S                   10000000     kernel32:KERNEL32.dll
 0000:ffff9000       .debug$S                   10000000     kernel32:KERNEL32.dll
 0000:ffff9000       .debug$S                   10000000     kernel32:KERNEL32.dll
 0000:ffff9000       .debug$S                   10000000     kernel32:KERNEL32.dll
 0000:ffff9000       .debug$S                   10000000     kernel32:KERNEL32.dll
 0000:ffff9000       .debug$S                   10000000     kernel32:KERNEL32.dll
 0000:ffff9000       .debug$S                   10000000     kernel32:KERNEL32.dll
 0000:ffff9000       .debug$S                   10000000     kernel32:KERNEL32.dll
 0000:ffff9000       .debug$S                   10000000     kernel32:KERNEL32.dll
 0000:ffff9000       .debug$S                   10000000     kernel32:KERNEL32.dll
 0000:ffff9000       .debug$S                   10000000     kernel32:KERNEL32.dll
 0000:ffff9000       .debug$S                   10000000     kernel32:KERNEL32.dll
 0000:ffff9000       .debug$S                   10000000     kernel32:KERNEL32.dll
 0000:ffff9000       .debug$S                   10000000     java:java.dll
 0001:0000057f       ?dllmain_crt_dispatch@@YGHQAUHINSTANCE__@@KQAX@Z 1000157f f   MSVCRT:dll_dllmain.obj
 0001:000005d2       ?dllmain_crt_process_attach@@YAHQAUHINSTANCE__@@QAX@Z 100015d2 f   MSVCRT:dll_dllmain.obj
 0001:000006d9       ?dllmain_crt_process_detach@@YAH_N@Z 100016d9 f   MSVCRT:dll_dllmain.obj
 0001:00000789       ?dllmain_dispatch@@YAHQAUHINSTANCE__@@KQAX@Z 10001789 f   MSVCRT:dll_dllmain.obj
 0001:00000894       ?dllmain_raw@@YGHQAUHINSTANCE__@@KQAX@Z 10001894 f   MSVCRT:dll_dllmain.obj
 0001:00000a03       ___get_entropy             10001a03 f   MSVCRT:gs_support.obj
 0001:00000afe       ?find_pe_section@@YAPAU_IMAGE_SECTION_HEADER@@QAEI@Z 10001afe f   MSVCRT:utility.obj
 0001:00000f60       $$000000                   10001f60     MSVCRT:sehprolg4.obj
 0002:000000f4       _GS_ExceptionPointers      100030f4     MSVCRT:gs_report.obj
 0002:000004c0       __sehtable$?dllmain_crt_process_attach@@YAHQAUHINSTANCE__@@QAX@Z 100034c0     MSVCRT:dll_dllmain.obj
 0002:000004e0       __sehtable$?dllmain_crt_process_detach@@YAH_N@Z 100034e0     MSVCRT:dll_dllmain.obj
 0002:00000508       __sehtable$?dllmain_dispatch@@YAHQAUHINSTANCE__@@KQAX@Z 10003508     MSVCRT:dll_dllmain.obj
 0002:00000528       __sehtable$___scrt_is_nonwritable_in_current_image 10003528     MSVCRT:utility.obj
 0002:00000550       .edata                     10003550     prefs.exp
 0002:00000578       rgpv                       10003578     prefs.exp
 0002:000005a4       rgszName                   100035a4     prefs.exp
 0002:000005d0       rgwOrd                     100035d0     prefs.exp
 0002:000005e6       szName                     100035e6     prefs.exp
 0002:000005f0       $N00001                    100035f0     prefs.exp
 0002:0000062f       $N00002                    1000362f     prefs.exp
 0002:00000671       $N00003                    10003671     prefs.exp
 0002:000006b1       $N00004                    100036b1     prefs.exp
 0002:000006f3       $N00005                    100036f3     prefs.exp
 0002:00000733       $N00006                    10003733     prefs.exp
 0002:00000773       $N00007                    10003773     prefs.exp
 0002:000007b2       $N00008                    100037b2     prefs.exp
 0002:000007f0       $N00009                    100037f0     prefs.exp
 0002:00000833       $N00010                    10003833     prefs.exp
 0002:00000876       $N00011                    10003876     prefs.exp
 0002:00000aaa       .idata$6                   10003aaa     advapi32:ADVAPI32.dll
 0002:00000ad8       .idata$6                   10003ad8     java:java.dll
 0002:00000c06       .idata$6                   10003c06     kernel32:KERNEL32.dll
 0002:00000c58       .idata$6                   10003c58     vcruntime:VCRUNTIME140.dll
 0002:00000d22       .idata$6                   10003d22     ucrt:api-ms-win-crt-heap-l1-1-0.dll
 0002:00000d42       .idata$6                   10003d42     ucrt:api-ms-win-crt-runtime-l1-1-0.dll
 0003:00000018       ?__proc_attached@@3HA      10004018     MSVCRT:dll_dllmain.obj
 0003:00000020       _GS_ExceptionRecord        10004020     MSVCRT:gs_report.obj
 0003:00000070       _GS_ContextRecord          10004070     MSVCRT:gs_report.obj
 0003:00000360       ?is_initialized_as_dll@@3_NA 10004360     MSVCRT:utility.obj
 0003:00000361       ?module_local_atexit_table_initialized@@3_NA 10004361     MSVCRT:utility.obj
 0003:00000364       ?module_local_atexit_table@@3U_onexit_table_t@@A 10004364     MSVCRT:utility.obj
 0003:00000370       ?module_local_at_quick_exit_table@@3U_onexit_table_t@@A 10004370     MSVCRT:utility.obj
 0004:00000060       $R000000                   10005060     prefs.dll.res
